:03005300020F7623
:0D000300EF7E0833D2939292C293DEF72273
:0D0010008F828E83E0FF120003A3DDF82233
:10001D008F828E837D00058690FF00E00586F0A31C
:0D002D00058690FF10E00586F0A3DDEA22B5
:050056007C05DCFE2228
:08005B00D290D2963090FD22F4
:10006300D290D291120056C291120056C290120041
:02007300562213
:10007500EF7E0833929112005612005B120056C2B1
:1000850090120056DEEDD29112005B120056A2913D
:03009500C29022F4
:10009800D2917E0812005B120056A29133C29012D0
:1000A8000056DEF0C29112005B120056C290D29147
:0500B800120056FF22BA
:1000BD00D2917E0812005B120056A29133C29012AB
:1000CD000056DEF0D29112005B120056C290D29112
:0500DD00120056FF2295
:10003A00C29112005612005B120056D2911200565B
:01004A002293
:101A6000534F554E4442415354415244204C4E52E0
:101A7000005625312E3366284329204156264856E4
:101A800044004D004100493243206572726F72205C
:101A90002D20736574005320005400412000253030
:101AA000325820202530325820202530325820202E
:011AB0000035
:1000E2009000001223120000000030081A90000055
:1000F2001222FA1223837F007E087D007C001221E7
:10010200C990000012230630091A9000001222FA48
:100112001223837F207E007D007C001221C9900083
:1001220000122306300A1A9000001222FA122383C8
:100132007F107E007D007C001221C99000001223F6
:100142000690000474A0F0E4900005F0A3F0A3046C
:10015200F0A37403F0A3742FF09000001222FA7837
:10016200081222A91223837FFF7E007D007C0012E9
:10017200225290000AEFF07FFF7E007D007C001289
:1001820023839000001222FA12225290000BEFF009
:10019200E4A3F09000001222FA78101222A912238E
:1001A200837F0F7E007D007C0012225290000DEFB3
:1001B200F01200637F3A1200757F68120075E490B6
:1001C200000EF0A3F090000EE0FEA3E0FFC3940A3D
:1001D200EE64809480501F74042FF582EE3400F593
:1001E20083E0FF12007590000FE004F070069000AB
:1001F2000EE004F080CF12003A900004740FF0A3D6
:1002020074CBF01200637F3A1200757F681200759A
:10021200E4900006F0A3F0900006E0FEA3E0FFC326
:100222009402EE64809480501F74042FF582EE34A1
:1002320000F583E0FF120075900007E004F07006FD
:0C024200900006E004F080CF12003A2289
:10024E009000101223067F4D7E3B7D807C00122392
:10025E00839000101222FA121C581223837FC17E43
:10026E00507D007C00121AD59000141223067F498F
:10027E007E007D007C001223839000141222FA125D
:10028E001BE01223837F3F7E007D007C00121AD577
:10029E00121CD41223837FFF7EFF7D0F7C0012225F
:1002AE005290001812230690001C74A0F0E49000E7
:1002BE001DF0A3F0A304F0A37403F0A3742DF0902B
:1002CE0000181222FA78081222A91223837FFF7EC9
:1002DE00007D007C00122252900022EFF07FFF7E04
:1002EE00007D007C001223839000181222FA122245
:1002FE0052900023EFF0E4A3F09000181222FA7847
:10030E00101222A91223837F0F7E007D007C001223
:10031E002252900025EFF01200637F3A1200757F93
:10032E0068120075E4900026F0A3F0900026E0FE1F
:10033E00A3E0FFC3940AEE64809480501F741C2FB8
:10034E00F582EE3400F583E0FF120075900027E091
:10035E0004F07006900026E004F080CF12003A7F81
:10036E004D7E2C7D447C001223839000101222FAC5
:10037E00121C581223837FC17E507D007C00121AFE
:10038E00D59000141223067F497E007D007C00125A
:10039E0023839000141222FA121BE01223837F3F54
:1003AE007E007D007C00121AD5121CD41223837F8E
:1003BE00FF7EFF7D0F7C0012225290001812230642
:1003CE0090001C74A0F0E490001DF0A3F0A304F0C4
:1003DE00A37403F0A3742EF09000181222FA78087A
:1003EE001222A91223837FFF7E007D007C00122241
:1003FE0052900022EFF07FFF7E007D007C001223E2
:10040E00839000181222FA122252900023EFF0E489
:10041E00A3F09000181222FA78101222A912238348
:10042E007F0F7E007D007C00122252900025EFF09F
:10043E001200637F3A1200757F68120075E4900017
:10044E0026F0A3F0900026E0FEA3E0FFC3940AEE90
:10045E0064809480501F741C2FF582EE3400F58357
:10046E00E0FF120075900027E004F0700690002661
:10047E00E004F080CF12003A90001C740FF0A374C9
:10048E00CBF01200637F3A1200757F68120075E49C
:10049E0090001EF0A3F090001EE0FEA3E0FFC394B8
:1004AE0002EE64809480501F741C2FF582EE34008F
:1004BE00F583E0FF12007590001FE004F0700690C7
:0B04CE00001EE004F080CF12003A2274
:1004D900900028EEF0A3EFF090002C7402F0A374C2
:1004E90000F0A37428F0A37402F0A37400F0A374BD
:1004F9002AF090002CE0FBA3E0FAA3E0F9900001B8
:1005090012212BFF90002FE0FBA3E0FAA3E0F9EF03
:1005190012215A90002CE0FBA3E0FAA3E0F9122182
:1005290010FF90002FE0FBA3E0FAA3E0F99000018F
:0D053900EF12216E90002AE0FEA3E0FF22E9
:1005460090003212230690003A7402F0A37400F071
:10055600A37432F0A37402F0A37400F0A37436F00F
:1005660090003AE0FBA3E0FAA3E0F9900003122121
:100576002BFF90003DE0FBA3E0FAA3E0F9EF122188
:100586005A90003AE0FBA3E0FAA3E0F990000212C9
:10059600212BFF90003DE0FBA3E0FAA3E0F99000D9
:1005A60001EF12216E90003AE0FBA3E0FAA3E0F916
:1005B60090000112212BFF90003DE0FBA3E0FAA37F
:1005C600E0F9900002EF12216E90003AE0FBA3E002
:1005D600FAA3E0F9122110FF90003DE0FBA3E0FA38
:1005E600A3E0F9900003EF12216E9000361222FA72
:0105F60022E2
:1005F700900040EBF0A3EAF0A3E9F0E4A3F0A3F046
:10060700900040E0FBA3E0FAA3E0F9122E3A900035
:1006170043E0FCA3E0FDC39FEE6480F8EC648098A0
:100627005026900040E0FBA3E0FAA3E0F98D828C0E
:100637008312212BFF120A39900044E004F0700660
:09064700900043E004F080B822A9
:10065000900045EFF0A3EBF0A3EAF0A3E9F0120A53
:100660002B90004AEFF0900045E0FF3395E0FEEF5D
:100670007803C333CE33CED8F9FF120A05E49000D5
:1006800049F0900049E0FFC36480948850229000B4
:1006900046E0FBA3E0FAA3E0F9EF3395E08F82F5A3
:1006A0008312212BFF120A39900049E004F080D216
:0D06B00090004AE0FF3395E0FE120A192287
:1006BD00C3EF64809480400FD3EF6480948E500715
:1006CD0090436DEFF080037F002290FF127430F0A5
:1006DD00E4FFFEFDFC90004BF0A3F0C3EF941EEE83
:1006ED00648094805025E4FCFDC3ED94C8EC6480D7
:1006FD009480501090004BE4F0A37402F00DED7057
:10070D00010C80E50FEF70010E80D090FF12743058
:10071D00F0E4FFFEFDFC90004BF0A3F0C3EF943C22
:10072D00EE648094805025E4FCFDC3ED94C8EC6428
:10073D00809480501090004BE4F0A37402F00DED06
:10074D0070010C80E50FEF70010E80D090FF1274D8
:10075D0030F0E4FFFEFDFC90004BF0A3F0C3EF94EE
:10076D001EEE648094805025E4FCFDC3ED94C8EC2E
:10077D0064809480501090004BE4F0A37402F00D4F
:10078D00ED70010C80E50FEF70010E80D090436D80
:10079D00E0FF60126403600EEF64066009EF640908
:1007AD006004EFB40C0890FF127430F0800690FFD7
:1007BD00127438F0E4FFFEFDFC90004BF0A3F0C383
:1007CD00EF941EEE648094805025E4FCFDC3ED94FF
:1007DD00C8EC64809480501090004BE4F0A3740238
:1007ED00F00DED70010C80E50FEF70010E80D090D3
:1007FD00FF127408F0E4FFFEFDFC90004BF0A3F037
:10080D00C3EF941EEE648094805025E4FCFDC3ED8F
:10081D0094C8EC64809480501090004BE4F0A37465
:10082D0002F00DED70010C80E50FEF70010E80D020
:10083D0090FF127401F0E4FFFEFDFC90004BF0A35D
:10084D00F0C3EF941EEE648094805025E4FCFDC34C
:10085D00ED94C8EC64809480501090004BE4F0A3AC
:10086D007402F00DED70010C80E50FEF70010E803C
:10087D00D090FF12740CF0E4FFFE90004BF0A3F04B
:10088D00A3F0A3F0C3EF941EEE648094805038E47F
:10089D0090004BF0A3F0C390004CE094C890004B37
:1008AD00E064809480501990004DE4F0A37402F040
:1008BD0090004CE004F0700690004BE004F080D600
:1008CD000FEF70010E80BD90FF127406F0E49000E2
:1008DD004BF0A3F0A3F0A3F0A3F0A3F090004BF026
:1008ED00A3F0C390004CE0941E90004BE064809404
:1008FD00805041E490004DF0A3F0C390004EE09481
:10090D00C890004DE064809480501990004FE4F041
:10091D00A37402F090004EE004F0700690004DE0DC
:10092D0004F080D690004CE004F0700690004BE08F
:07093D0004F080AE7F0122EF
:0D09440090FF12E030E7037F01227F0022C8
:10095100120944EF70FA90FF127401F0E4FFFEFDFA
:10096100FC900051F0A3F0C3EF941EEE64809480DC
:100971005025E4FCFDC3ED94C8EC648094805010D4
:10098100900051E4F0A37402F00DED70010C80E5CC
:080991000FEF70010E80D0226F
:10099900120944EF70FA90FF127402F0E4FFFEFDB1
:1009A900FC900053F0A3F0C3EF941EEE6480948092
:1009B9005025E4FCFDC3ED94C8EC6480948050108C
:1009C900900053E4F0A37402F00DED70010C80E582
:0809D9000FEF70010E80D02227
:1009E100AE07120944EF70FAEE5403440490FF126B
:0209F100F022F2
:1009F300AE07120944EF70FAEE5407440890FF1251
:020A0300F022DF
:100A0500AD07AC06120944EF70FAED543F4440902F
:040A1500FF12F022BA
:100A1900AD07AC06120944EF70FAED448090FF125D
:020A2900F022B9
:0E0A2B00120944EF70FA90FF12E0547FFF2290
:0E0A3900AE07120944EF70FA90FF13EEF022A0
:100A470090FF0E7404F090FF01E0FF90FF0EE4F0BA
:0F0A570090FF07E020E7F990FF07E030E6F92273
:0B0A6600EFC454F024A090FF06F02223
:06004B0090FF0EE03322DD
:100A7100900055EBF0A3EAF0A3E9F0A3E0F9A3E0BD
:100A8100FAA3E0904369C9F0A3EAF0A3E9F090FF6B
:100A910007E020E7F9900055E0FBA3E0FAA3E0F9B5
:100AA10090000112212BC454F024A090FF06F09075
:100AB100FF07E020E7F990FF07E030E6F9900055E5
:100AC100E0FBA3E0FAA3E0F990000212212B90FFD2
:100AD10001F090000312212B90FF02F09000081208
:100AE100212B90FF03F090000712212B90FF04F0BF
:100AF10090000612212B90FF05F090000512212B8A
:100B010024A0FF90000112212BC454F02FFF90006C
:100B11000412212B75F040A42F90FF06F012211032
:100B210090FF07F090FF07E020E7F990FF0EE0202B
:100B3100E7F990FF07E07814F630E30F900058E0F2
:0C0B4100A3E0FAA3E0AE02FF12001D22A8
:100B4D009000697420F0A3EFF0E4A3F0A304F0A3E8
:100B5D00F090005FE090006EF0900060E090006F0C
:100B6D00F0900061E0900070F0900062E0900071F4
:100B7D00F0900063E0F9A3E0FAA3E0900058C9F00B
:100B8D00A3EAF0A3E9F0900066E0F9A3E0FAA3E090
:100B9D0090005BC9F0A3EAF0A3E9F07B027A00793B
:050BAD0069120A71222B
:100BB200900072EEF0A3EFF0A3EDF0E075F010A458
:100BC200FF900073E024AEFD900072E03401CD2F5F
:100BD200FFED35F0FAA9077B02122110900075F0A3
:100BE200900074E075F010A4FF900073E02FFF9066
:100BF2000072E035F0FEEF24AFFDEE3401FAA905F4
:100C0200122110900076F0EF24B0FFEE3401FAA921
:100C120007122110900077F0900074E075F010A494
:100C2200FF900073E02FFD900072E035F0FCED24A0
:100C3200B1FFEC3401FAA907122110FF900078E409
:100C4200F0A3EFF0900077E0FB54C0FFC4131354FD
:100C520003FE900079E02400F0900078E03EF0EB93
:100C6200543F900077F0ED24B2FFEC3401FAA9076B
:100C72007B0212211090007AF0900074E075F0105F
:100C8200A4FF900073E02FFF900072E035F0FEEFBA
:100C920024B3FDEE3401FAA90512211090007BF075
:100CA200EF24B4FFEE3401FAA90712211090007C60
:100CB200F0900074E075F010A4FF900073E02FFD37
:100CC200900072E035F0FCED24B5FFEC3401FAA996
:100CD20007122110FF90007DE4F0A3EFF090007C5A
:100CE200E0FB54C0FFC413135403FE90007EE024C3
:100CF20000F090007DE03EF0EB543F90007CF0ED80
:100D020024B6FFEC3401FAA9077B021222BC900040
:100D12008712230690008BEBF0A37400F0A3748774
:100D2200F0A3EBF0A37400F0A3747FF090008BE0CB
:100D3200FBA3E0FAA3E0F990000312212BFF90003D
:100D42008EE0FBA3E0FAA3E0F9EF12215A90008BA8
:100D5200E0FBA3E0FAA3E0F990000212212BFF903E
:100D6200008EE0FBA3E0FAA3E0F9900001EF12216C
:100D72006E90008BE0FBA3E0FAA3E0F99000011271
:100D8200212BFF90008EE0FBA3E0FAA3E0F9900094
:100D920002EF12216E90008BE0FBA3E0FAA3E0F9D0
:100DA200122110FF90008EE0FBA3E0FAA3E0F9907D
:100DB2000003EF12216E900074E075F010A4FF9012
:100DC2000073E02FFF900072E035F0CF24BACF34E9
:100DD20001FAA9077B021222BC9000871223069017
:100DE200008EEBF0A37400F0A37483F090008BE00C
:100DF200FBA3E0FAA3E0F990000312212BFF90007D
:100E02008EE0FBA3E0FAA3E0F9EF12215A90008BE7
:100E1200E0FBA3E0FAA3E0F990000212212BFF907D
:100E2200008EE0FBA3E0FAA3E0F9900001EF1221AB
:100E32006E90008BE0FBA3E0FAA3E0F990000112B0
:100E4200212BFF90008EE0FBA3E0FAA3E0F99000D3
:100E520002EF12216E90008BE0FBA3E0FAA3E0F90F
:100E6200122110FF90008EE0FBA3E0FAA3E0F990BC
:0D0E72000003EF12216E7B027A00797522D9
:100E7F00A20BE433FF120A669002947420F0E4A3ED
:100E8F00F0A3F0A304F0A3F0E4A3F0A3F0A3F0A366
:100E9F00F09000587402F0A37400F0A37494F0A3C0
:100EAF00E4F0A3F0A3F07B027A027994120A717E28
:100EBF00007F947D01120BB2C003C002900091E03D
:100ECF00FBA3E0FAA3E0F8AC02AD03D002D0037E9F
:100EDF00007F121220DE7E007F947D02120BB2C0C3
:100EEF0003C002C001900091E0FBA3E0FAA3E0244D
:100EFF0012F9E43AA801FCAD03D001D002D0037E71
:100F0F00007F121220DE7E007F947D03120BB2C091
:100F1F0003C002C001900091E0FBA3E0FAA3E0241C
:100F2F0024F9E43AA801FCAD03D001D002D0037E2E
:100F3F00007F121220DE7E007F947D04120BB2C060
:100F4F0003C002C001900091E0FBA3E0FAA3E024EC
:100F5F0036F9E43AA801FCAD03D001D002D0037EEC
:070F6F00007F121220DE22B8
:100F7600C0E0C0F0C083C082C0D0C000C001C002C3
:100F8600C003C004C005C006C007E4FFFEFDFC9018
:100F9600029DF0A3F0C3EF9414EE64809480502574
:100FA600E4FCFDC3ED94C8EC64809480501090027C
:100FB6009DE4F0A37402F00DED70010C80E50FEFD7
:100FC60070010E80D090FF18E090436CF090436E55
:100FD6007401F0904361E0FBA3E0FAA3E0F9EA496B
:100FE60060031224355391BFD007D006D005D00434
:100FF600D003D002D001D000D0D0D082D083D0F0A0
:03100600D0E03205
:1010090090436CE024FE602324FE602624FC6029C2
:1010190024F8602C24F0602F24E0603224C060356D
:10102900247F70379003607401F02290036074028A
:10103900F0229003607407F0229003607408F02294
:101049009003607405F0229003607406F022900307
:0C105900607403F0229003607404F02225
:10106500E490029FF0A3F0538EF843A8809043616B
:101075007405F0A37410F0A37409F0E490436EF0C6
:1010850043E8047F011206BD7F041209F3120951DA
:101095007B057A1A79601205F77F407E00120A19DE
:1010A5009043727405F0A3741AF0A37471F0A3123F
:1010B5002312B6F37D3F7B027A0279A11224F97BD4
:1010C500027A0279A11205F7E4FFFEFDFC90032CDC
:1010D500F0A3F0C3EF94A0EE6480948F5025E4FC58
:1010E500FDC3ED94C8EC64809480501090032CE40B
:1010F500F0A37402F00DED70010C80E50FEF7001A7
:101105000E80D0120951E4FFFE120A197B057A1AE6
:1011150079821205F790032C7401F0E4A3F0120014
:10112500637F3A1200757F6A120075E490032EF012
:10113500A3F090032EE0FEA3E0FFC39402EE6480CB
:101145009480501F742C2FF582EE3403F583E0FF55
:1011550012007590032FE004F0700690032EE00452
:10116500F080CF12003AE490032CF0A3F012006354
:101175007F3A1200757F6A120075E490032EF0A382
:10118500F090032EE0FEA3E0FFC39402EE6480948A
:1011950080501F742C2FF582EE3403F583E0FF1287
:1011A500007590032FE004F0700690032EE004F024
:1011B50080CF12003A7B057A1A79841205F79002DE
:1011C5009FE07002A3E07009C208C209D20A1200AA
:1011D500E290029FE07002A3E0700B7F4B7E5A7D88
:1011E5007A7C6412024E90029FE07002A3E0600ECA
:1011F5001209517B057A1A79861205F780FE7B055F
:101205007A1A79961205F77B057A1A79841205F709
:1012150012004B40FB120A477B057A1A7999120591
:10122500F7E4FF90005F12231200000000900063B6
:101235007402F0A37403F0A37461F0A3E4F0A3F0C7
:10124500A3F0120B4D9005271222FA9003151223D5
:10125500069003151222FA1205469003151223066D
:1012650090052B1222FA90031912230690031912E6
:1012750022FA12054690031912230690031512222D
:10128500FA90005F1223069000637402F0A37403C2
:10129500F0A37461F0A3E4F0A3F0A3F0FF120B4DEB
:1012A50090036FE0FEA3E0FF90031DEEF0A3EFF0C7
:1012B5001204D990031DEEF0A3EFF0900371E090B6
:1012C5000323F09003851222FA90031F1223069040
:1012D500031F1222FA12054690031F1223069003DC
:1012E50023E0FFE4FCFDFE12238390031F1222FA84
:1012F5001221F012238390031DE0FEA3E0FFE4FC1E
:10130500FD1221C99003241223069003191222FA13
:0F1315009003281223067B057A1A799B1205F79D
:101324001209517F417E00120A197F3E120A397F49
:1013340020120A397F58120A397F20120A397F2075
:10134400120A397F2D120A397F2B120A397F201293
:101354000A397F20120A397F2D120A397F2B120A8B
:10136400397F20120A397F20120A397F2D120A3957
:101374007F2B120A399003607402F0900324122226
:10138400FA9003091223069003281222FA90030DFF
:1013940012230690030D1222FA90033412230690AE
:1013A40003091222FA1216E353E8FB900360E014D7
:1013B40070030216B524FD7003021468147003024E
:1013C40014D114700302155A1470030215C3147057
:1013D4000302164C240560030216DC7F007E017DA7
:1013E400007C001223839003581222FA1221DC900D
:1013F40003581223069003581222FA900309122369
:10140400069003241222FA1223839003091222FA6B
:10141400122284500C9003241222FA9003091223FE
:10142400069003281222FA1223839003091222FA47
:10143400122284600E400C9003241222FA900309B5
:101444001223069003607401F043E80490030D1224
:1014540022FA9003341223069003091222FA121678
:10146400E30213AC9003581222FA1223837F007E06
:10147400017D007C001221C99003581223069003B9
:10148400581222FA9003091223069003281222FA12
:101494001223839003091222FA122284600E400C54
:1014A4009003281222FA9003091223069003607411
:1014B40001F043E80490030D1222FA90033412233E
:1014C400069003091222FA1216E30213AC7F007E7F
:1014D400007D017C001223839003581222FA12210A
:1014E400DC9003581223069003581222FA90030941
:1014F4001223069003241222FA1223839003091262
:1015040022FA122284500C9003241222FA90030926
:101514001223069003281222FA122383900309123D
:1015240022FA122284600E400C9003241222FA90B4
:1015340003091223069003607401F043E804900346
:071544000D1222FA9003349E
:10154B001223069003091222FA1216E30213AC902F
:10155B0003581222FA1223837F007E007D017C0048
:10156B001221C99003581223069003581222FA90A5
:10157B0003091223069003281222FA1223839003E5
:10158B00091222FA122284600E400C9003281222B8
:10159B00FA9003091223069003607401F043E804E8
:1015AB0090030D1222FA90033412230690030912B2
:1015BB0022FA1216E30213AC7F007E007D007C0141
:1015CB001223839003581222FA1221DC9003581233
:1015DB0023069003581222FA900309122306900354
:1015EB00241222FA1223839003091222FA12228464
:1015FB00500C9003241222FA900309122306900335
:10160B00281222FA1223839003091222FA1222843F
:10161B00600E400C9003241222FA90030912230649
:10162B009003607401F043E80490030D1222FA90CA
:10163B0003341223069003091222FA1216E3021343
:10164B00AC9003581222FA1223837F007E007D0098
:10165B007C011221C99003581223069003581222C1
:10166B00FA9003091223069003281222FA122383FD
:10167B009003091222FA122284600E400C90032868
:10168B001222FA9003091223069003607401F043AF
:10169B00E80490030D1222FA9003341223069003F0
:1016AB00091222FA1216E30213AC9003581222FA13
:1016BB0090030912230643E80490030D1222FA90BB
:1016CB0003341223069003091222FA1216E30213B3
:0816DB00AC43E8040213AC2249
:1016E3009003301223069003301222FA900358120B
:1016F30023069043647403F0A37461F0F9A37402A6
:10170300F0A37403F0A3E9F090035C12231200002A
:1017130000009043727405F0A3741AF0A3749EF052
:101723007F007E007D007CFF1223839003581222EA
:10173300FA12225278181222A9904375EEF0A3EF01
:10174300F07F007E007DFF7C0012238390035812FC
:1017530022FA12225278101222A9904377EEF0A3B4
:10176300EFF07F007EFF7D007C00122383900358FF
:101773001222FA12225278081222A9904379EEF02B
:10178300A3EFF07B027A0379381224F97F067E00F7
:10179300120A197B027A0379381205F79003301283
:1017A30022FA9003581223069003341222FA1223CA
:1017B300839003581222FA1222844003021A5F9084
:1017C3000360E064016003021A5F7FFFFEFDFC1209
:1017D30023839003581222FA1222521223837F008A
:1017E3007E007D007C00122284600302187B9043FC
:1017F300727405F0A3741AF0A3749EF07F007E0048
:101803007D007CFF1223839003581222FA12225286
:1018130078181222A9904375EEF0A3EFF07F007EB3
:10182300007DFF7C001223839003581222FA1222B8
:101833005278101222A9904377EEF0A3EFF07F00C5
:101843007EFF7D007C001223839003581222FA123C
:10185300225278081222A9904379EEF0A3EFF07B8D
:10186300027A0379381224F97F067E00120A197B63
:10187300027A0379381205F77F407E007D007C00F1
:1018830012238390035C1222FA122284500302195A
:1018930060E59020E762904366E0FBA3E0FAA3E0F3
:1018A300F9C003C002C001904364E0FEA3E0FFF966
:1018B300D082D083D0E064027008E965827003EEC1
:1018C300658360347D40120010904365E02440F04E
:1018D300904364E03400F0C3A3E09461FF90436459
:1018E300E09403FEEF7003EE644070A590436474CC
:1018F30003F0A37461F08099904364E0FEA3E0FFDA
:10190300AA06F97B02C003C002C001A3E0A3E0FA68
:10191300A3E0F9C3D082D083D0E0E99582EA95832E
:101923004013904366E0A3E0A3E0C39FFFEA9EFE5B
:10193300E4FCFD8022904366E0A3E0FAA3E0FFC34A
:10194300904365E09FFF904364E09AFEC3E49FFFEA
:1019530074409EFEE4FCFD90035C1223067F007E30
:101963003E7D007C0012238390035C1222FA122234
:101973008440030217AB53E8FB9003581222FA90FA
:10198300005F122306904366E0F9A3E0FAA3E09018
:101993000063C9F0A3EAF0A3E9F0A3E4F0A3F0A382
:1019A300F0FF120B4D43E804904367740275F00097
:1019B300122192904366E0A3E0FAA3E0C39461FF8F
:1019C300EA9403FEEFB40012EEB4400E9043667443
:1019D30002F0A37403F0A37461F0904364E0FEA3E8
:1019E300E0FFAA06F97B02C003C002C001A3E0A383
:1019F300E0FAA3E0F9C3D082D083D0E0E99582EA8C
:101A030095834013904366E0A3E0A3E0C39FFFEAFE
:101A13009EFEE4FCFD8022904366E0A3E0FAA3E08F
:101A2300FFC3904365E09FFF904364E09AFEC3E4E5
:101A33009FFF74409EFEE4FCFD90035C122306901E
:101A430003581222FA1223837F017E007D007C005B
:061A53001221C9900358A6
:071A59001223060217AB2265
:03000000021AB130
:061AB10075814D02106575
:101AB700DA0CD902800BD906300701B35005021D95
:101AC700899207021D75D9F680F9D2068002C206EF
:101AD700121DBA300606C86002B207C89206DAD0ED
:101AE700D9E4B8000A121E01A2069207021D5E6021
:101AF700FBB54500400F121E01A20692F7A20792FE
:101B070006A2F79207C398F40424E740DF2419AD2F
:101B170041AC40AB3F7A00C394084008CDCCCBFA28
:101B2700E4CD80F424086010F9C3ED13FDEC13FC39
:101B3700EB13FBEA13FAD9F1A206300701B34030E1
:101B47008A49E5422BF54AE5433CF54BE5443DF52B
:101B57004C501A13F54CE54B13F54BE54A13F54A70
:101B6700E54913F5490545E54570020546021D148B
:101B7700E4C39AF549E5429BF54AE5439CF54BE5F5
:101B8700449DF54C500DB207C378497F04E496F69F
:101B970008DFFA7A047019E545C39408F545500241
:101BA7001546E4C549C54AC54BF54CDAE8021DB5EB
:101BB70020E7BAE5457002154615457849C37F0405
:081BC700E633F608DFFA80E8BE
:101BCF00DA03B80003021D89D9028002D9F7021D7A
:101BDF0075121DBA300701B392077004D9E780055B
:101BEF00DADEB80003021DB5D9E2C3947E500215A8
:101BFF00462545F545500205467847760008B84D0D
:101C0F00FA783F7947E608FAE8FC78428AF0E60866
:101C1F00A427F709E5F037F7500989F00907E760BE
:101C2F00FBA9F0B845E61919ECF8B842D8021D1413
:101C3F00021DA0B8FFFA021D89D9FB021D75DAF645
:101C4F00B800F0021DB5122265121DBA300701B39C
:101C5F0092077007D9E3B800E280DBDAE1B800023F
:101C6F0080E1D9D5C8C39850021546247F5002058C
:101C7F0046F545784C76007A1A7B80C3E542953F4E
:101C8F00E5439540E54495414016C3E542953FF540
:101C9F0042E5439540F543E5449541F544E64BF65F
:101CAF00DA03021D14EB03FB30E703187600C3E5DC
:101CBF004233F542E54333F543E54433F54440CA37
:051CCF0030E7DD80B6E6
:101CD400EF8EF0A2F7D2F73392D5C3947F5006E487
:101CE400FFFEFDFC229420400474FF80F304CCFE2C
:101CF400E4FFFAE5F0CC6012C3CC13CCCD13CDCE07
:101D040013CECF13CF0450EEDAEC30D5D7022276BF
:10249100E5082472F582E43443F583E005082290CF
:1024A100436F301303904372E475F00112234C0221
:1024B1002110200CE97F2ED20C8018EF540F2490AC
:1024C100D43440D4FF30100BEF24BFB41A005003B2
:1024D1002461FFE50960021509050CE50C70020590
:1024E1000B20145930130E90436FE475F001122341
:1024F1004CEF02215A022CAD7403D2138003E4C2C3
:1025010013F50890436F12237AE4F509F50BF50CE6
:10251100E50960077F201224D480F5F50AC20DC2B7
:102521000CC20EC20FC211C212C2141224A0FF703B
:102531000D3013057F001224E8AF0CAE0B22B42539
:1025410050C2D5C2101224A0FF24D0B40A00501EDC
:1025510075F00A20D50DC509A42509F5097002D227
:102561000F80E0D20CC50AA4250AF50A80D524CF34
:10257100B41A00EF5004C2E5D2100227BED20D807A
:10258100C0D20C80BCD20E80B8D2D580B6122491B4
:10259100FF1224D4022511D21280A6D21180A212D8
:1025A1002491FB122491FA122491F94A4B70067975
:1025B100B07A287B05200E33E509602FAF0ABF00F2
:1025C100011F7E008E8275830012212B60050EEEA5
:1025D1006F70F1C2D5EBC0E0EAC0E0E9C0E0EE12F5
:1025E100281AD0E0F9D0E0FAD0E0FB122110FF6008
:1025F100A3EBC0E0EAC0E0E9C0E01224D4D0E024BB
:1026010001F9D0E03400FAD0E0FBE50A60DDD50A3B
:10261100DA8081D20E809E1227FE60F7E50A121E33
:1026210017A90A600BE50A12289DEF7003D50AF578
:10263100EA30E702F404C3995079EAF4250A043038
:10264100E701E404F50A800D1227FE60C6EA050AD7
:10265100250A121E17EA90439EF030E701E4250A8D
:1026610004D50A042011011412281AE4C0E012282A
:102671009D90439EE0601320E70714F01224BC8074
:102681002204F0D0E014C0E07F001224BCE50A600F
:10269100071224B3150A800B3011031224B3D0E0C2
:1026A100022511D0E00480C41227FE609EE50A04D1
:1026B100121E1790439EEAF0E50A04201102600100
:1026C10004240412281A74FF04C0E012289D122465
:1026D100BCE50A20110260031224B3D0E0B50AE878
:1026E1007F451224C690439EE07F2B30E7047F2D67
:1026F100F404C0E01224D4D0E075F00A84C0F012D2
:1027010024BDD0E01224BD0225117910800C790876
:0E2711008008D2D5790A8006790AC2D5C21294
:10271F00E4FAFDFEFF122491FC7B08200D13122416
:10272F0091FD7B10300C0A122491FE122491FF7B35
:10273F0020EC3382D592D55013C3E4300C069FFFA3
:10274F00E49EFEE4200D039DFDE49CFCE4CBF8C267
:10275F000DEC700CCFCECDCCE824F8F870F38017C9
:10276F00C3EF33FFEE33FEED33FDEC33FCEB33FB06
:10277F00994002FB0FD8E9EB300D05F8D0E0C448C3
:10278F00B20DC0E00AEC4D4E4F78207B0070C2EACC
:10279F00C0E012281CD0F0D0E0200D04C4C0E0C46B
:1027AF00B20DC0F01224BDD0F0D5F0EB02251112FE
:1027BF00240F25A053270B5825824C257E42270F27
:1027CF004F271344271349258E432719552649466A
:1027DF0026A94526184728C25025862D258A2E253D
:1027EF00982B259C2325882028BD2A000025921090
:1027FF000C03750A06122491FC122491FD122491E8
:10280F00FE122491FF904397021E54790AA2D520FD
:10281F000F14301109B910020404B9080104A2D52C
:10282F00201202500104200E61920EB509005032A1
:10283F00C0E07F20300F177F30A20E72127211503E
:10284F000D122871C20EC212C2117F30800F3011CB
:10285F0003E9C0E01224D4301103D0E0F9D0E0B581
:10286F0009CE3011177F30B9100C1224D47F583095
:10287F0010077F788003B908031224D4300E057F28
:10288F002D0224D47F2B2012F822920E80D47F00A9
:10289F00B40700500B2497F582E43443F583E0FF2F
:1028AF0022286E756C6C29002D4958504443D21460
:1028BF00022542122491B406004001E49028B793F8
:1028CF001224C5743A1224C5D20F75090402270BBE
:1028DF00E50D30180104F8232824A2F582E43443CF
:1028EF00F5832290439F3018039043A2E475F001C3
:1028FF0012234C022110C5117002151014C511209E
:10290F00180660DEFF022D2F90439F74FFF5F00233
:10291F002363FF022D37E50E6006D50E037F0022DD
:10292F000511E51170020510201803022D1B9043AD
:10293F009FE475F00112234C122110FF2212292F50
:10294F00EFC0E0122921D0E040F380AAD218800214
:10295F00C21890439F12237AE4F50FF50DF510F589
:10296F0011750E00C217C215C216C2191228F2FF36
:10297F007005AF0F7E0022B425301228F2FF24D04D
:10298F00B40A00500C75F00AC50EA4250EF50E8082
:10299F00E924CFB41A00EF5002C2E5022B97D216EA
:1029AF0080D8D21580D4D21980D0EF1229215005AA
:1029BF0012294C80ACEFC0E012292FD0E06F60A13C
:1029CF00EF606A12290580AA7401C50E6002F50E28
:1029DF0012292FEF605720190E1228DFE475F0012E
:1029EF0012234CEF12215AD50EE6201904050D05BE
:1029FF000F80C0E50E6002050E12294C122925EF3B
:102A0F00602BC0E0122921D0E05004122905E4FF09
:102A1F0020190E1228DFE475F00112234CEF12215A
:102A2F005AEF70D8201904050D050F808630180451
:102A3F00E4122905E50F60030229817EFF7FFF2243
:102A4F00E50E6002050E12294CD21BD21A1229254F
:102A5F00EF301B0260D7C0E0122905D0E0122BE344
:102A6F00500712292FC21A80E4201913201A0520AB
:102A7F000002050F1228DF122343050D1222DE027A
:102A8F0029707910803FEF122905790880371229B4
:102A9F004C12292FEF6096BF301712292FEF608D40
:102AAF00BF780280DDBF58DE12294C12292FEF604C
:102ABF00E4790AEFB42D04D2178019B42B028014D5
:102ACF00122905790AE50E6002050EE9C0E0122908
:102ADF004CD0E0F9D21AE4FCFDFEFFE9C0E012236E
:102AEF0083122925EFF81223B4D0F0E8604DB461BA
:102AFF00004007B47B005002C2E524D0503DFA24B9
:102B0F00F6500724F95034240AFAEAB5F000502B96
:102B1F00CFA9F0A42FFF92D5E9C5F0CEA4A2D53E40
:102B2F00FE92D5E9C5F0CDA4A2D53DFD92D5E9C55C
:102B3F00F0CCA4A2D53CFCC21A80A0E8C0E02019BA
:102B4F002A201A08050F3017031222761228DF12D7
:062B5F002343050D2015C3
:102B65000B20160DEE8FF01221A880091222DE80AF
:102B750004EF12215AD0E0122905022970201910FC
:102B85001228DF122343050DE5108511F01221A847
:102B950080E812240F2A02532A915829B14C29ADF5
:102BA5004229AD482A994F2AB74429D7432A9D4936
:102BB5002AD2552A4F462A4F452A4F4729B52A2B4F
:062BC500824E000029B958
:101D1400E54C20E7137849C37F04E633F608DFFA7D
:101D2400E545700215461545E54933784A7F03E6D3
:101D34003400F6500E08DFF7754C800545E5457014
:101D4400020546E54620E7547027E545604E0460E9
:101D540020854C44854B43854A425320F0AC42AD28
:101D640043A207E54513FFE54492E7FEA845022395
:101D7400BCE4F544F543F542F5467545FF5320F0C0
:101D840043200580D874FFF544F543F542754600B9
:101D9400F545D2075320F043200980C15320F04376
:101DA4002003E4F544F543F542F546F545C20780C2
:061DB400AC5320F080ECAE
:101DBA0079017A018544F0E545A2F7339207754621
:101DCA0000F5456002D2F785F044A845B8FF080936
:101DDA00E544C2E76001098C3F8D408EF0A2F7EF1F
:101DEA003304700A0AC2F705F00AD5F0011A146022
:071DFA0002D2F785F041223F
:101E0100C88845C544C541C544C543C540C543C54A
:061E110042C53FC542225C
:101E1700F920E73624F950037907E4F42402FBE5B7
:101E270082158270021583DBF6E024FB501BE96004
:101E370014E4F0E582158270021583E004F0B40A19
:0D1E470008E4F0D9EE7401F00A22C2D522A1
:101E5400EE33EF3392D5FB602AB4FF33EEC2E77B57
:101E64000560067A1E7979E4227A1E798220D504E7
:101E74007A1E797D224E614E002B494E46002D4933
:101E84004E4600E47A08F0A3DAFC7B0074072212C1
:101E94002383EBFF75F010A4FAABF08FF0744DA41C
:101EA4002BFBACF050010CC3EA94F0FAEB943AFB30
:101EB400EC9426FCE544C2E7FF75F056A4F4241420
:101EC400C5F0F434C58FF0A42AE5F03BE43CF020DF
:101ED400E70B121FDC1223E6121C58800BF40412C9
:101EE4001FDC1223E6121BE0EE33EF33C39482406F
:101EF40009704EEED2E794A050471223BCE0FAEEEC
:101F0400A2E7D2E7FEEF332482FBE4C3CC33CCCD8B
:101F140033CDCE33CE33DBF3F0A37B078CF0740ADE
:101F2400A4FCAFF08DF0740AA42FFDAFF050010FA4
:101F34008EF0740AA42FFEE435F0F0A3DBDE740700
:101F440022E004F020E708121FDC121C5880AEF4D3
:091F540004121FDC121BE080A442
:102BCB00C21CC21DC21EC21FF9E4F512FCFDFEFFA2
:102BDB00122383E9C082C083D083D082101BE120F3
:102BEB001E0DB42D05D21ED3E473B42B0280F82432
:102BFB00D050429409503C240A301F13F8D0F07483
:102C0B000AA42872E7404FC5F0704BC0F080D8D2B1
:102C1B001DFCE4121F78122265122383E4FCFD7E57
:102C2B00207F41121BE0121AD5122383301CB815DA
:102C3B001280B4240A201F2FB4FE07201C29D21C9B
:102C4B0080A524EB600424E0701DA21E921CD21FF1
:102C5B00C21EC0E080915320F043200974FFFCFD9D
:102C6B00FEFF1223BC8038E4301F0BD0E0301E0275
:102C7B00F404A21C921E301DDD251220D2D8A2E72F
:102C8B00921F5002F404B4260050CB121FDC201FFD
:102C9B0005121BE08003121C58301E03121F5DC36C
:022CAB00E473D0
:101F5D00EE33EF33600C047005EE547F7004EFB276
:031F6D00E7FF2269
:101F70007920800C7910800479087D007E007F0034
:101F80003392D530D503122276EC33400FEF33FF76
:101F9000EE33FEED33FDEC33FCD9EE22EECCF5F062
:0C1FA000747E29A2D513FF92F7AEF02248
:101FAC000000803F000020410000C84200007A443D
:101FBC0000401C460050C347002474498096184BBF
:101FCC0020BCBE4CCA1B0E5A1CC25367AEC59D74B6
:101FDC00FB6006540760142323121FFDEB5438607A
:101FEC002A122383121FF7121BE022EB543803240E
:101FFC001CAA83A982901FACFF93FCEFA393FDEF67
:0C200C00A393FEEFA393FF8A8389822236
:10201800E709F608DFFA8046E709F208DFFA803EAA
:1020280088828C83E709F0A3DFFA8076E309F60853
:10203800DFFA806EE309F208DFFA806688828C8313
:10204800E309F0A3DFFA805A89828A83E0A3F608BD
:10205800DFFA804E89828A83E0A3F208DFFA8042A1
:1020680080AE80B480BA80C480CA80D080DA80E430
:1020780080378023805389828A83ECFAE493A3C84B
:10208800C582C8CCC583CCF0A3C8C582C8CCC583DB
:10209800CCDFE9DEE7800D89828A83E493A3F60822
:1020A800DFF9ECFAA9F0EDFB2289828A83ECFAE0E9
:1020B800A3C8C582C8CCC583CCF0A3C8C582C8CC88
:1020C800C583CCDFEADEE880DB89828A83E493A3D8
:1020D800F208DFF980CC88F0ED14B4040050C32472
:1020E8001E83F582EB14B4050050B72415832582AE
:1020F800F582EF4E60ACEF60010EE58290206873C8
:08210800000402000C060012A5
:10211000BB020689828A83E0224003BB0402E722D5
:0B212000400789828A83E49322E322B7
:10212B00BB020CE58229F582E5833AF583E0224078
:10213B0003BB0406E92582F8E622400DE58229F56A
:0F214B0082E5833AF583E49322E92582F8E222C4
:10215A00BB020689828A83F0224003BB0402F7226B
:04216A005001F3220B
:10216E00F8BB020DE58229F582E5833AF583E8F0A6
:10217E00224003BB0406E92582C8F6225005E92554
:04218E0082C8F222EF
:10219200C5F0F8A3E028F0C5F0F8E58215827002D8
:0621A2001583E038F02275
:1021A800BB020A89828A83F0E5F0A3F0224003BBD0
:1021B8000406F709A7F019225006F3E5F009F31908
:0121C80022F4
:1021C900EF2545FFEE3544FEED3543FDEC3542FC88
:0321D9000223BC22
:1021DC00C3EF9545FFEE9544FEED9543FDEC95421E
:0421EC00FC0223BC12
:1021F000EFF88545F0A4FFE545C5F0CEF9A42EFE25
:10220000E435F0CDFA88F0E544A42EFEED35F0FD7E
:10221000E433CC8545F0A42CFCE5448AF0A42CFCE6
:10222000E54389F0A42CFCE54288F0A42CFC89F05D
:10223000E544A42DFDEC35F0FCE54388F0A42DFD2C
:10224000EC35F0FC8AF0E545A42DFDEC35F0FC0200
:0222500023BCAD
:10225200EF5545FFEE5544FEED5543FDEC5542FC6E
:032262000223BC98
:10226500CFC545CFCEC544CECDC543CDCCC542CCDB
:012275002246
:0E227600C3E49FFFE49EFEE49DFDE49CFC2279
:10228400C3EF9545F8EE954448F8ED954348F8ECCE
:10229400954248F892D5D082D0831223B4E8A2D5CF
:0522A400C083C082228E
:1022A900E8600FECC313FCED13FDEE13FEEF13FF13
:0322B900D8F12237
:1022BC00BB020789828A830222FA4003BB0405E928
:1022CC00F8022451400789828A83022469E9F802C2
:0222DC00245D7F
:1022DE00BB020789828A830223064003BB0405E9F9
:0C22EE00F8022479400122E9F80224855E
:0C22FA00E0FCA3E0FDA3E0FEA3E0FF2257
:0C230600ECF0A3EDF0A3EEF0A3EFF0224A
:10231200A8828583F0D083D0821223291223291226
:102322002329122329E473E493A3C583C5F0C5834B
:10233200C8C582C8F0A3C583C5F0C583C8C582C815
:012342002278
:09234300E0FBA3E0FAA3E0F9229B
:10234C00F8E0FBA3A3E0F925F0F0E582158270021A
:07235C001583E0FA38F022BE
:10236300F8E0FBA3A3E025F0F9F0E5821582700203
:072373001583E038FAF022A7
:09237A00EBF0A3EAF0A3E9F02264
:10238300E54D054D6022232324B0C082C083F5822E
:10239300E43443F583E542F0A3E543F0A3E544F0D9
:1023A300A3E545F0D083D0828F458E448D438C4284
:1023B30022AF45AE44AD43AC42E54D146022232326
:1023C300C082C08324B0F582E43443F583E0F54250
:1023D300A3E0F543A3E0F544A3E0F545D083D08221
:0323E300154D2273
:1023E600E54D6024232324B0C082C083F582E43403
:1023F60043F583E542F0A3E543F0A3E544F0A3E506
:0924060045F0D083D082054D227F
:10240F00D083D082F8E4937012740193700DA3A35C
:10241F0093F8740193F5828883E473740293686070
:06242F00EFA3A3A380DF70
:062435008A838982E47332
:102CAD00EFB40A07740D122CB8740A309811A89954
:102CBD00B8130CC2983098FDA899C298B811F63087
:072CCD0099FDC299F599225F
:102CD400904434EBF0A3EAF0A3E9F0904434E0FB31
:102CE400A3E0FAA3E0F91221106018904434E0A3A1
:102CF400E475F00112243BA9F0FA122110FF122C02
:0D2D0400AD80D87F0A122CAD7E007F00222A
:0A2D11003098FDAF99C2987E0022B1
:102D1B0010200B122D11BF0D027F0A022CAD904417
:042D2B0037E0FF226C
:082D2F00904437EFF0D220229E
:102D3700EFC394094006EFC3940E4005EF6420707B
:062D470003D38001C3224A
:102D4D00904438EBF0A3EAF0A3E9F0A3ECF0A3ED87
:102D5D00F0E4A3F0A3F090443CE024FFFF90443B4B
:102D6D00E034FFFEC390443EE09FEE6480F8904453
:102D7D003DE06480984003022E1F122D1B904438B5
:102D8D00E0FBA3E0FAA3E0F990443DE0FCA3E0FDF5
:102D9D00F5828C83EF12216EEF640A6075904438D2
:102DAD00E0FBA3E0FAA3E0F98D828C8312212B6462
:102DBD0008702590443DE07002A3E0600E90443E03
:102DCD00E024FFF090443DE034FFF07F20122CAD65
:102DDD007F08122CAD022D63904438E0FBA3E0FA7E
:102DED00A3E0F990443DE0FEA3E0F5828E8312212D
:102DFD002BFF64117003022D63EF64137003022D1A
:102E0D006390443EE004F0700690443DE004F0020F
:102E1D002D63904438E0FBA3E0FAA3E0F990443D24
:0D2E2D00E0FEA3E0F5828E83E412216E2208
:102E3A0090443FEBF0A3EAF0A3E9F0E4FFFE9044EC
:102E4A003FE0FBA3E475F00112243BA9F0FA12213A
:0B2E5A001060070FEF70010E80E422F3
:10243B00A3F8E0C5F025F0F0E58215827002158354
:06244B00E0C838F0E822B1
:0C245100E6FC08E6FD08E6FE08E6FF22B7
:0C245D00E2FC08E2FD08E2FE08E2FF22BB
:10246900E493FCA3E493FDA3E493FEA3E493FF2286
:0C247900ECF608EDF608EEF608EFF6228F
:0C248500ECF208EDF208EEF208EFF22293
:00000001FF
